:1000000000308A003C280000831A0A28A500030E4D
:10001000A6000F288312A500030EA600A6140A0846
:10002000AD008A018313A50E0408A7002008A800CC
:100030002108A9002208AA002308AB002408AC006C
:1000400083128C308400001C27280C18582827089D
:1000500084002808A0002908A1002A08A2002B0873
:10006000A3002C08A4002D088A00260E830083120A
:10007000250EA61883160900FF2383169000003072
:100080008A003A2A0A108A100A118207403457342B
:100090002234063415340C34083456340034043415
:1000A000FF340A108A100A11820702340134043422
:1000B000EC308F009A308E00273085003F3087006B
:1000C000000000003108023C031CB1012E30310752
:1000D0008400000887002E30310784000008403972
:1000E000A0000310200CD70031085120073A570414
:1000F0008500B10A0C108A11272807309900831651
:10010000050803308312A000A00B842819088C1165
:100110001F1300300838831691001F129F161F17F7
:1001200083129F171F1418308316850027308312FF
:100130008500831687013730831287008530900051
:10014000EC308F009A308E00C0308B0483160C1474
:1001500083124A2A3830840000080319BE2801306F
:10016000A100A001A00BB228A10BB1284A30A00029
:10017000A00BB82800000000800BAF280034A001BD
:10018000A101A201A301D001D101D201D3014F08E5
:100190004E044D044C040319FD282030D4000310F4
:1001A000C80DC90DCA0DCB0DD00DD10DD20DD30D7B
:1001B0004F085302031DE6284E085202031DE6288D
:1001C0004D085102031DE6284C085002031CF72875
:1001D0004C08D0024D08031C4D0FD1024E08031CE1
:1001E0004E0FD2024F08031C4F0FD3020314A00D71
:1001F000A10DA20DA30DD40BCF2800005030840018
:1002000000342030D000CC01CD01CE01CF01470811
:10021000A3004608A2004508A1004408A00003105E
:10022000201C20294808CC0749080318490FCD078E
:100230004A0803184A0FCE074B0803184B0FCF0785
:10024000CF0CCE0CCD0CCC0CA30CA20CA10CA00C92
:10025000D00B0F290034C701C601C5011E30C400F0
:100260003F08CB003E08CA003D08C9003C08C80052
:1002700001212308C7002208C6002108C500200864
:10028000C4002308CB002208CA002108C9002008A6
:10029000C800CF01CE012730CD00F630CC00BF2002
:1002A0002308C8002208C7002108C6002008C5008E
:1002B000A0002108A1002208A2002308A300200812
:1002C0004220A100AE002E08403C031D6929FF30EA
:1002D000AE00C701C601C5011E30C4003F08CB00F7
:1002E0003E08CA003D08C9003C08C8000121230897
:1002F000C7002208C6002108C5002008C400230842
:10030000CB002208CA002108C9002008C800CF017C
:10031000CE012730CD00F630CC00BF200008C00051
:10032000840A0008C100840A0008C200840A000888
:10033000C300C701C601C5010A30C4004308CB0091
:100340004208CA004108C9004008C800012123082A
:10035000C7002208C6002108C5002008C4002308E1
:10036000CB002208CA002108C9002008C800CF011C
:10037000CE012730CD00F630CC00BF202308C800C6
:100380002208C7002108C6002008C500A0002108D7
:10039000A1002208A2002308A30020084220A100F7
:1003A000AF00C701C601C5010A30C4004308CB0035
:1003B0004208CA004108C9004008C80001212308BA
:1003C000C7002208C6002108C5002008C400230871
:1003D000CB002208CA002108C9002008C800CF01AC
:1003E000CE012730CD00F630CC00BF200008C00081
:1003F000840A0008C100840A0008C200840A0008B8
:10040000C300C701C601C5010A30C4004308CB00C0
:100410004208CA004108C9004008C8000121230859
:10042000C7002208C6002108C5002008C400230810
:10043000CB002208CA002108C9002008C800CF014B
:10044000CE012730CD00F630CC00BF202308C800F5
:100450002208C7002108C6002008C500A000210806
:10046000A1002208A2002308A30020084220A10026
:10047000B000902A84011F3083051F1300308316BB
:1004800091000730831299007F30AE00AF00B000BA
:10049000B1017D28B601B501B401B301B701370838
:1004A000133C031C712A0C30A1001F08C33921041E
:1004B0009F000130B800AA209F149F185D2A831660
:1004C0001E088312B3071E0803181E0FB40700305E
:1004D00003180130B507003003180130B607B70A1A
:1004E0004F2A3608CB003508CA003408C900330843
:1004F000C800CF01CE01CD011430CC00BF202308AD
:10050000BB002208BA002108B9002008B80023085F
:10051000BF002208BE002108BD002008BC002B2916
:0A052000C830B800AA204A2A630080
:0207FE00443481
:02400E00C431BB
:00000001FF
